:1000000044C01895189518957FC21895189518959D
:100010001895D1C218951895189518951895189592
:100020001895EEEDEBE7DEDDDBD7BEBDBBB77E7D21
:100030007B774F4E00004F464600414D0000504D2B
:1000400000002D2D2D3C53657420486F75723E2D98
:100050002D2D00002D2D3C536574204D696E757457
:10006000653E2D2D00002D2D3C5365742020416CE4
:1000700061726D3E2D2D00002D2D2D3C5365742099
:10008000446174653E2D2D2D00000FE50DBF02E08B
:100090000EBF00E009BF03E003BF02EC02BF03E0B4
:1000A00004BB08E002BD002704BD05E005BD02B5A4
:1000B00007700730E1F301E409BF0FEF07BB789445
:1000C0001FEF0027602E702E6AD163D12227C1E076
:1000D0006627552744270027902EC02EA02EB02E2D
:1000E00071E081E090E055D12227F0E0E2E4C8958C
:1000F000002049F0283011F400EC8ED1002DA1D160
:1001000031962395F4CF222701E0702E00E070167F
:1001100039F00DE10615D1F7CAD2ADD1C130B1F732
:1001200000E0702E0DE1061511F4C1D2A4D1BD3E40
:1001300041F401E0702E6395683109F0E7CF60E08B
:10014000E5CFB73E49F401E0702E6A956F3F09F0A4
:10015000DDCF67E1DBCF60E0BE3E09F0B9F619D133
:100160002227F0E0E4E5C895002049F0283011F49A
:1001700000EC52D1002D65D131962395F4CF222782
:1001800001E0702E01E0702E00E0701639F00DE1F4
:100190000615D1F78CD26FD1C130B1F700E0702EC7
:1001A0000DE1061511F483D266D1BD3E41F401E0A4
:1001B000702E53955C3309F0E7CF50E0E5CFB73EA2
:1001C00049F401E0702E5A955F3F09F0DDCF5BE303
:1001D000DBCF50E0BE3E09F0B9F6DBD02227F0E0DD
:1001E000E8E7C895002049F0283011F400EC14D15C
:1001F000002D27D131962395F4CF222701E0702ED0
:1002000000E0701639F00DE10615D1F750D233D168
:10021000C130B1F700E0702E0DE1061511F447D2A0
:100220002AD1BD3E51F401E0702E73957D3011F05E
:10023000D4D1E6CF71E0D1D1E3CFB73E59F401E09C
:10024000702E7A95703011F0C8D1DACF7CE0C5D12C
:10025000D7CF71E0BE3E09F099F601E0702EBDD116
:1002600000E0701639F00DE10615D1F720D203D168
:10027000C130B1F700E0702E0DE1061511F417D270
:10028000FAD0BD3EC1F401E0702E8395803281F03A
:100290008F3141F4743061F0763051F0793041F0B3
:1002A0007B3031F08D3111F4723011F096D1D8CF0E
:1002B00081E093D1D5CFB73EC9F401E0702E8A9585
:1002C000803011F08AD1CCCF743061F0763051F0AB
:1002D000793041F07B3031F0723011F48CE103C0A1
:1002E0008FE101C08EE179D1BBCF81E0BE3E09F044
:1002F000B7CF01E0702E00E0701639F00DE1061561
:10030000D1F7D5D1B8D0C130B1F700E0702E0DE1F2
:10031000061511F4CCD1AFD0BD3E51F401E0702EE2
:100320009395943611F059D1E6CF90E056D1E3CFB2
:10033000B73E59F401E0702E9A959F3F11F04DD1D0
:10034000DACF93E64AD1D7CF90E0BE3E09F0D3CFC3
:1003500044D101E0702E00E0701639F00DE1061571
:10036000D1F7A5D188D0C130B1F700E0702E0DE1F2
:10037000061519F432D19BD17ED0BE3E09F4B3CE1E
:10038000BE3D09F404D2BE3719F401E09026702E68
:10039000E2CF01E041D003E0102F6AD0089500E0E1
:1003A00002BB0FEF01BB0FE0102F62D003E002BBD6
:1003B0000000949A000094980FE0102F59D003E0A9
:1003C00002BB0000949A000094980FE0102F50D0C8
:1003D00003E002BB0000949A000094980FE0102FF5
:1003E00047D002E002BB0000949A0000949800E21B
:1003F00013D00CE011D006E00FD0089500EF01BB40
:10040000959A9698949A0000949830B2949A000025
:10041000949833FCF7CF08950F93F0DF0FEF01BBF3
:100420000F910F9302950F7002BB0000949A000089
:1004300094980F910F7002BB0000949A000094985A
:1004400008950F93DBDF0FEF01BB0F910F93029520
:100450000F7002BB969A0000949A000094980F9136
:100460000F7002BB969A0000949A00009498089529
:100470001123F1F70895C13031F0C23061F0C3307B
:1004800091F0C430B1F01DD0A03011F4BB27089515
:100490004A2EC2E0089515D0A41519F4BA2FC3E06E
:1004A0000895C1E008950DD0AB1709F40895C4E094
:1004B000089507D0AB1711F4C3E00895BB27C1E03E
:1004C00008950FE00ABB00EF0BBB00000000000026
:1004D000000000000000000000000000000000001C
:1004E00009B3A02F00EF0ABB0FE00BBB0000000018
:1004F00000000000000000000000000000000000FC
:10050000000009B3A02B08955FB60F93EF93FF93FC
:1005100002E04395C0264C33B9F5442753955C332C
:1005200099F555276395683179F56627839580326B
:1005300019F4739581E024C08F3161F4743039F07F
:10054000763029F0793019F07B30D1F401F07395D1
:1005500081E016C08E3129F4723091F4739581E0F8
:100560000FC08D3169F4723059F4F92FF03041F039
:10057000F43031F0F450F3360AF4F8CF739581E09B
:100580007D3011F471E09395092D013049F4A616E0
:1005900061F4B51651F445301AF403E0C02E05C0DD
:1005A00002E0C02202E0C026C026C5BAFF91EF914A
:1005B0000F915FBE18955FB60F93EF93FF931A9557
:1005C00002EC02BF01E0600E0EE1601609F4662441
:1005D000FF91EF910F915FBE1895DBDE0027EAE0F7
:1005E000F72EFE1611F0FE1618F00395FE1AF9CF3D
:1005F000E0E30E0F26DF0027E1E0FE1611F0FE1605
:1006000018F00395FE1AF9CFE0E30E0F1ADF00276A
:100610000FE217DF0027EAE0F82EFE1611F0FE16B3
:1006200018F00395FE1AF9CFE0E30E0F0ADF00275A
:10063000E1E0FE1611F0FE1618F00395FE1AF9CF50
:10064000E0E30E0FFEDE00270FE2FBDE0027EAE00C
:10065000F92EFE1611F0FE1618F00395FE1AF9CFCA
:10066000E0E30E0FEEDE0027E1E0FE1611F0FE16CD
:1006700018F00395FE1AF9CFE0E30E0FE2DE002733
:1006800001E0901699F400ECC7DE00E2DADE0AE23F
:10069000D8DE01E4D6DE0CE4D4DE01E4D2DE02E5ED
:1006A000D0DE0DE4CEDE0AE2CCDE08950895002708
:1006B000EAE0E62EEE1611F0EE1618F00395EE1AAB
:1006C000F9CF006708BB14E0D3DE0027E1E0EE16A7
:1006D00011F0EE1618F00395EE1AF9CF006B08BB77
:1006E00014E0C6DE00270027EAE0E52EEE1611F042
:1006F000EE1618F00395EE1AF9CF006D08BB14E062
:10070000B7DE0027E1E0EE1611F0EE1618F00395C3
:10071000EE1AF9CF006E08BB14E0AADE0895002798
:10072000EAE0EA2CEE1611F0EE1618F00395EE1A38
:10073000F9CF006708BB14E09BDE0027E1E0EE166E
:1007400011F0EE1618F00395EE1AF9CF006B08BB06
:1007500014E08EDE00270027EAE0EB2CEE1611F005
:10076000EE1618F00395EE1AF9CF006D08BB14E0F1
:100770007FDE0027E1E0EE1611F0EE1618F003958B
:10078000EE1AF9CF006E08BB14E072DE089501DEA8
:100790002227F0E0E6E6C895002049F0283011F461
:1007A00000EC3ADE002D4DDE31962395F4CF222762
:1007B00000E0A02E01E0702E00E0701639F00DE18F
:1007C0000615D1F7ACDF57DEC130B1F700E0702E6F
:1007D0000DE1061511F4A3DF4EDEBD3E59F401E034
:1007E000702E01E0A00E08E1A01609F0E5CF00E0B0
:1007F000A02EE2CFB73E69F401E0702E01E0A01A0E
:100800000FEFA01609F0D8CF07E1A02ED5CF002713
:10081000B02EBE3E09F081F60027B02E01E0702E0A
:1008200000E0701639F00DE10615D1F778DF23DE10
:10083000C130B1F700E0702E0DE1061511F46FDF45
:100840001ADEBD3E59F401E0702E01E0B00E0CE35B
:10085000B01609F0E5CF0027B02EE2CFB73E69F41D
:1008600001E0702E01E0B01A0FEFB01609F0D8CFFA
:100870000BE3B02ED5CF0027B02EBE3E09F081F697
:0808800001E0702E902E089596
:00000001FF
